:0200000480007A
:100000006F00C004732F2034930F8000630AFF0336
:10001000930F90006306FF03930FB0006302FF038A
:10002000170F0080130F0FFE63040F0067000F000F
:10003000732F203463540F006F004000136E9E53E3
:10004000171F00002320CFFD6FF09FFF732540F1A5
:100050006310050073251030635805000F00F00F82
:10006000130E100073000000130E00009702000032
:10007000938282F973905230735020307350303035
:1000800073504030970200809382C2F7638C020065
:10009000739052109302B01A739022307323203061
:1000A000E39E62F873500030970200009382420191
:1000B00073901234732540F17300203097200000B4
:1000C000938040F483910000930EF00F130E2000F4
:1000D000639CD125972000009380C0F2839120007B
:1000E000930E00F0130E30006390D125972000008E
:1000F000938040F183914000B71E0000938E0EFF65
:10010000130E40006392D12397200000938080EF6C
:1001100083916000B7FEFFFF938EFE00130E500028
:100120006394D12197200000938020EE8391A0FF5B
:10013000930EF00F130E60006398D11F97200000FC
:100140009380A0EC8391C0FF930E00F0130E70001B
:10015000639CD11D97200000938020EB8391E0FFEA
:10016000B71E0000938E0EFF130E8000639ED11BFE
:1001700097200000938060E983910000B7FEFFFFA5
:10018000938EFE00130E90006390D11B9720000009
:10019000938040E7938000FE83910002930EF00F5E
:1001A000130EA0006392D11997200000938080E580
:1001B0009380B0FF83917000930E00F0130EB00097
:1001C0006394D117130EC0001302000097200000A3
:1001D000938060E38391200013830100B71E000029
:1001E000938E0EFF6312D3151302120093022000A8
:1001F000E31E52FC130ED0001302000097200000F3
:10020000938080E08391200013000000138301009D
:10021000B7FEFFFF938EFE006318D3111302120086
:1002200093022000E31C52FC130EE00013020000B6
:1002300097200000938000DD8391200013000000D0
:100240001300000013830100930E00F0631ED30D12
:100250001302120093022000E31C52FC130EF00064
:1002600013020000972000009380E0D983912000C2
:10027000B71E0000938E0EFF6398D10B130212007D
:1002800093022000E31052FE130E0001130200003F
:1002900097200000938040D7130000008391200036
:1002A000B7FEFFFF938EFE006390D1091302120088
:1002B00093022000E31E52FC130E100113020000F3
:1002C00097200000938000D413000000130000006A
:1002D00083912000930E00F06398D1051302120061
:1002E00093022000E31E52FC97210000938181D1EC
:1002F0000391010013012000930E2000130E200132
:100300006314D103972100009381C1CF03910100B1
:100310001300000013012000930E2000130E300183
:100320006314D101631CC0010F00F00F63000E00C5
:10033000131E1E00136E1E00730000000F00F00F4E
:10034000130E100073000000731000C000000000C6
:10035000000000000000000000000000000000009D
:10036000000000000000000000000000000000008D
:10037000000000000000000000000000000000007D
:040380000000000079
:1010000000000000000000000000000000000000E0
:1010100000000000000000000000000000000000D0
:1010200000000000000000000000000000000000C0
:1010300000000000000000000000000000000000B0
:081040000000000000000000A8
:10200000FF0000FFF00F0FF00000000000000000D4
:040000058000200057
:00000001FF
